:0300000002128B5E
:03000B000200C12F
:03002B000203CB02
:03005B0002059803
:0300730002058EF5
:1000800002030406080C10182030406080020304AC
:1000900006080C101820304080FF0406080C1018C9
:1000A0002030406080A0C000000001010003020277
:1000B000010D0D040206020D0505050D06030502DE
:1000C00002C2AFC0D0C0E0205A0D302F02E473301E
:1000D000600280F90203B7306306C294C292C290F4
:1000E00085258AC25AE525F4700221AA056130608F
:1000F00013206A19758B00D0E0D0D0C294C292C28E
:1001000090D2AF32C294C292C29002019AD26EC211
:100110006FE565601CC3E5611495654014C26ED23D
:100120006FC3E5619564500302019A756100020195
:100130009A206C14C294C292C2907401D5E0FDD290
:1001400095D293D29102019AC294C292C290E53D97
:1001500020E22520E10D207502D295307502D29162
:1001600002019A20E005D29302019A207502D291F1
:10017000307502D29502019A20E11520E00D20751C
:1001800002D295307502D29102019AD29302019A5D
:10019000207502D291307502D295758B00D0E0D0D7
:1001A000D0C294C292C290D2AF32D0E0D0D0D2AFFF
:1001B0003261B7E525600A207502D294307502D20B
:1001C00090C29261B7E5256002D292207502C2907A
:1001D000307502C29461B7E525600A207502D2909D
:1001E000307502D294207502C294307502C29061BB
:1001F000B7207502C295307502C291E525600A20CC
:100200007502D294307502D290207502C291307579
:1002100002C295C29261B7207502C295307502C2C2
:1002200091207502C291307502C2957428D5E0FD07
:10023000E525600A207502D294307502D290C292F0
:1002400061B7207502C295307502C291E525600A3A
:10025000207502D294307502D290C293C29261B7D7
:10026000207502C295307502C291C2937428D5E000
:10027000FDE525600A207502D294307502D290C245
:100280009261B7C293E5256002D292207502C295B1
:10029000307502C291207502C290307502C294611D
:1002A000B7C293207502C295307502C2917428D5E9
:1002B000E0FDE5256002D292207502C29030750201
:1002C000C29461B7C293E5256002D292207502C242
:1002D00091307502C295207502C290307502C294A9
:1002E00061B7C293207502C291307502C29574281D
:1002F000D5E0FDE5256002D292207502C2903075EE
:1003000002C29461B7207502C291307502C295E5B0
:1003100025600A207502D290307502D294C29320D3
:100320007502C294307502C29061B7207502C29105
:10033000307502C295C2937428D5E0FDE525600AA8
:10034000207502D290307502D294207502C294308A
:100350007502C29061B7207502C291307502C295D4
:10036000E525600A207502D290307502D29420757E
:1003700002C295307502C291207502C29430750296
:10038000C29061B7207502C291307502C295207586
:1003900002C295307502C2917428D5E0FDE5256052
:1003A0000A207502D290307502D294207502C29450
:1003B000307502C29061B7E525F4F58A758B00753A
:1003C0006000D25AD0E0D0D0D2AF32C2AFC0D0C0DD
:1003D000E0D2D3C2CEE528600A741F552E604915BD
:1003E00028812878007900E580307601F430E40235
:1003F00078FF53DACF20760343DA2030760343DAEE
:1004000010C2D8C269E580307601F430E40279FF89
:10041000C3E89970CE305903752840741F552E607B
:10042000037528408858D268E52960041529813B66
:10043000741F552E600543DA01C2D820680281C0BE
:10044000E558F8C268741F552E60367982B70431BA
:10045000C3E894F0400374F0F8E8C4540F28F87926
:1004600084B703028181C313C3138721200802C309
:0E04700013200A06C3C898F8818128F85003AB
:10047E0074FFF8C3E8955F5003E55FF8E52C54066A
:10048E007030882230630AC3E522955C4003855C98
:10049E00227882B6041CC3E5229524401278A096D9
:1004AE00400DE52426F52450097524FF0204C0856D
:1004BE00222420CF09D0E0D0D0C2D3D2AF32C2CFC7
:1004CE007801E5286008741F552E70021528C3E5C3
:1004DE005894014005755B0081EFE55B04600205F1
:1004EE005B7982B7020EE548601EC3E52294324066
:1004FE00178547227982B7030FE548600BC3E522C3
:10050E0094324004798E8722C3E5239522600840F9
:10051E00041523A1250523D8C80562E562700215CE
:10052E0062D563537563017803C3E562941E404739
:10053E00C3E562946450087801756303020559C3DC
:10054E00E562949650057801756301C3E55D9524C7
:10055E004018E548701485245DE5620460037562F9
:10056E001E75630175233C020585C3E55D285005A4
:10057E00755DFFA185F55DD0E0D0D0C2D3D2AF328C
:10058E00C2AF53917FC258D2AF32C2AFC0D0C0E01B
:10059E00C0F0D2D3A8FBA9FCC2D8306902A1FB538C
:1005AE00DACF20760343DA1030760343DA20D269AD
:1005BE00E580307601F420E402A1CF88268927E178
:1005CE009B53DACF20760343DA2030760343DA10DA
:1005DE00C2D8C269741F552E7002E1817800E58081
:1005EE00307601F430E402E1818858E18153DACFAC
:1005FE0020760343DA2030760343DA10C26920599D
:10060E0002C1B553DACF20760343DA1030760343B6
:10061E00DA20C2D8D26988538954C3E89551F8E9D3
:10062E009552F9E4FB7AFAC3E894C8E994005008AD
:10063E00E4D2E4FB7A0AC188C3E89468E9940150D5
:10064E0008E4D2E3FB7A0FC188C3E894D0E99402A0
:10065E005008E4D2E2FB7A1EC188C3E894A0E99464
:10066E00055008E4D2E1FB7A3CC188C3E89498E9CE
:10067E0094085006E4D2E0FB7A78C3E89555FCE97D
:10068E009556FD30E708ECF42401FCEDF4FD7557AA
:10069E00007008C3EC9A500375570188558956A807
:1006AE0053A95488518952C3E89526F8E99527F93C
:1006BE00307402E154307302E154307202E14DE9BC
:1006CE00C313F9E813F8307102E14DE9C313F9E8E9
:1006DE0013F8307002E14DE9C313FDE813FC205905
:1006EE0018C3EC941CED94024003020781ED7009CF
:1006FE00C3EC94C8500302079B74002077037896CE
:10070E00E624FAFEE43400FFC3EC9EFCED9FFD50A0
:10071E000678007900E154C3EC94FFED9400400696
:10072E0078FF7900E154EC856CF0A4C5F0A2F733A4
:10073E00F87900400302077078FF7900020770E92C
:10074E00C313F9E813F830740EE9600278FFC3E8BA
:10075E001338F8E43400F9C3E894FFE9940040023A
:10076E0078FF8858D268205902E181741FF4552E03
:10077E004BF52E752840741F552E700375280A30C0
:10078E005902E19B741F552E600353DAFE75292022
:10079E00741F552E700375290AD0F0D0E0D0D0C248
:1007AE00D3D2AF327901E1CA7903E1CA790AE1CA3B
:1007BE00791EE1CA7964E1CA79C8E1CA7817E4D52D
:1007CE00E0FDD8FAD9F6227A147B780207F17A1076
:1007DE007B8C0207F17A0D7BB40207F17A0B7BC892
:1007EE000207F1AC257525017902B275E4C293D5E5
:1007FE00E0FDE5256002D292D5E0FDC292D5E0FD86
:10080E00D293D5E0FDE525600A207502D2943075AD
:10081E0002D290E56DD5E0FD207502C294307502CE
:10082E00C2907496D5E0FDD9C1EAF8D5E0FDD8FBAB
:10083E00DBB1C2938C2522C37C007D0075F00005D0
:10084E00F0EA33FAEB33FB50F6EB13FBEA13FAC381
:10085E00E9FFE8FEE89AF8E99BF95004EFF9EEF8A3
:0F086E00B3EC33FCED33FDD5F0DFEDF9ECF82200
:10087D00E889F08A20D2D4F8A9F07B0030F70B7B01
:10088D00FFF42401F8E9F43400F9E88520F0A4AD73
:10089D00F0F8E98520F0A4AFF0FEED2EF974003FDD
:1008AD00FA7C04C3EA13FAE913F9E813F8DCF48BC4
:1008BD00F030F70AE8F42401F8E9F43400F9E88996
:1008CD00F0C2D4F8A9F0227882B60403020960C3FD
:1008DD00E55894014018E54870377805C37994B709
:1008ED0002027812C3E53B9400E53C984020E548B0
:1008FD006009855E5D7562FF756301852224E4F5EF
:10090D003FF540F541F542F543F54802096075485C
:10091D0001C37994E79402601BE523F43333F91393
:10092D00F8E9540104F9E854FEC39440F8E9940041
:10093D00F902095CE523F433333333F913F8E95441
:10094D00070404F9E854F8C39440F8E99400F988D1
:10095D003F894022E548603BC3E53C13F9E53B1375
:10096D00F8C3E53F98F8E54099F9500CC3E8948039
:10097D00E994FF401602099CC3E8947FE994005066
:10098D000302099C787F790002099C788079FF88A1
:10099D0044894522E5486058E5442541F8E545354B
:1009AD0042F9854520E4300701F43543FA30E70973
:1009BD00C3EA94F040150209DEC3EA940F50030216
:1009CD0009DE78FF79FF7A0F0209DE780079007A67
:1009DD00F0C3E524955C5006E524600921F7E54553
:1009ED0020E70D21F7E54530E706884189428A4326
:1009FD0022E5487003020A61789EE6FAC3E54433A6
:100A0D00F8E54533F9117DE930E70BC3E89480E94A
:100A1D0094FF40134138C3E8947FE994005002419C
:100A2D0038787F79004138788079FFE820E715C361
:100A3D00E52398F84009C3E894014003020A5F7862
:100A4D0001020A5FE8F424012523F84003020A5F3E
:100A5D0078FF884622E5487003020AC3789FE6FABC
:100A6D00A842A943117DE930E70CC3E89401E9944C
:100A7D00FF4016020A9AC3E894FFE994005003025E
:100A8D000A9A78FF7900020A9A780179FFE920E73E
:100A9D0015C3E54698F84009C3E894014003020ADE
:100AAD00C17800020AC1E8F424012546F84003028A
:100ABD000AC178FF8824227883E6F520121002758A
:100ACD00E890E5E820ECF0A8BDA9BE12109A756873
:100ADD0085756900C3740013FD748513FC74852C32
:100AED00FC74003DFDECFAEDFBC3E89AE99B401464
:100AFD00E5682485F568E5693400F569EA2CFAEBBB
:100B0D003DFB80E5AE68AF69C3E56913F9E5681390
:100B1D00F8C3E913F9E813F8E56828F566E56939CE
:100B2D00F5677A03C3E913F9E813F8DAF7AA201A7F
:100B3D007009756800756900020B581AEA6008EEB5
:100B4D0028FEEF39FFDAF88E688F692275E890225A
:100B5D007883E6FFE5E820ECF7A8BDA9BE056AC3DA
:100B6D00E56A94084052756A00E97007E56B601BF1
:100B7D00020B8CC3E8956B6010E56B5006600C148E
:100B8D00020B980460F9020B98E56BF56BC3946D3D
:100B9D00F84021755CC0C3E89404F84017755C807B
:100BAD00C3E89404F8400D755C40C3E89404F84024
:100BBD0003755C0075BB0E22EFC39401601BC3E887
:100BCD0094FFE994035012C3E89568E995695009BB
:100BDD00E55C600C155C020BEDE55CF46002055CF8
:100BED00A85CC3E524985002A8248825C3E5259563
:100BFD005D400B855D25E55DF46003855D5CC3E5BA
:100C0D006AB4070375BB102230610278323062027C
:100C1D007850E52C5406601FE879A187F0A4C5F043
:100C2D00A2F733F8C3E8955C4002A85C88228824BB
:100C3D008825306102885E22788FE6FFC3EF940528
:100C4D005018C3EF94045020C3EF94035028C3EF02
:100C5D0094025030C3EF940150387533A075340FA2
:0E0C6D0075353C75360581AD7533C075341292
:100C7B0075354075360681AD75337075341775351E
:100C8B00D075360781AD75334C75341D7535C4750C
:100C9B00360981AD7533287534237535B875360B28
:100CAB0081AD85334F853450753B00753C0822A8C8
:100CBB004FA950020CC5A849A94A759100C3E498E5
:100CCB00F594E499F595759104D25875C820A8CC84
:100CDB00A9CD75C824AA39AB3A8839893AC3E89AA1
:100CEB00F8E99BF9AA3BAB3CC3EB13FDEA13FCC33E
:100CFB00ED13FDEC13FCC3EA9CFAEB9DFBEA28FA1F
:100D0B00EB39FB8A3B8B3C400122753BFF753CFF6B
:100D1B0022305802A11C759100C3E4954BF594E465
:100D2B00954CF595759104D258227892E6FF7E107A
:100D3B00305B027F053063047F037E00A93CA83B38
:100D4B007A04C3E913F9E813F8DAF7C3E89EF8E974
:100D5B009400F94009C3E89402E994005004780226
:100D6B00E4F9E9FBE8FAC3E913FDE813FCC3EF94DC
:100D7B0003602EEF20E00DE82CF8E93DF9ECFAEDDD
:100D8B00FB020D99E828F8E939F97A02E4FBC3EF85
:100D9B009403400D8A4D8B4E8849894A8C4B8D4C60
:100DAB0022884D894E8A498B4A8C4B8D4C22305868
:100DBB0002A1B9759100C3E4953BF594E4953CF51C
:100DCB0095759104D25822753E00752000020DE1F5
:100DDB00753E00752040D2AF053E20580122759D0F
:100DEB0000E53CC313C313F8086030306A06C31325
:100DFB00C313F808C3E8940A4002780A306D08C39D
:100E0B00E8940440027804C3E53C9408400D759DBA
:100E1B0002C3E53C94104003759D03205803D2AFE9
:100E2B0022793C206D027914D2AF0000C2AF205A58
:100E3B000A7928206D02790D306FE03063027978E2
:100E4B00C3E58B9940D5E59BF4F45440B52002A142
:100E5B00E1D8C8D2AF22C25B789CE6146007E53EAE
:100E6B00147002D25B30630B0538205810753800B4
:100E7B00020E88205807158115810217D92275910A
:100E8B0000C3E4954DF594E4954EF595759104D218
:100E9B005822AE25305B4F78A3E6FFBF010BD25C27
:100EAB00752500C294C292C290B121305C037525A6
:100EBB0000305802C1B6BF020BD25C752500C2943C
:100ECB00C292C29078A2B6010DB121305C03752598
:100EDB0000305802C1D6BF030BD25C752500C294FB
:100EEB00C292C290D189305C03752500305802C183
:100EFB00F1305B04C25C8E2522C2AFC293206A0321
:100F0B00020F26900305206C12306E0F207502C263
:100F1B0091307502C2957428D5E0FD207502D295EB
:100F2B00307502D291759F70753D02D2AF22C2AF60
:100F3B00206A03020F5B9002C4306E17C2932075B8
:100F4B0002C291307502C2957428D5E0FD020F5E86
:100F5B009001C5207502C290307502C294305A06BA
:100F6B00E5256002D292207503759F0030750375DD
:100F7B009F20753D03D2AF22C2AF207502C29530C0
:100F8B007502C291206A03020FA5900283206C0A9E
:100F9B00306E07C2937428D5E0FD207502D29130D4
:100FAB007502D295207503759F20307503759F00D0
:100FBB00753D04D2AF22C2AF206A03020FE3900249
:100FCB0042306E17207502C295307502C291C293E2
:100FDB007428D5E0FD020FE69001B3C292305A0E91
:100FEB00E525600A207502D294307502D290759F68
:100FFB0070753D05D2AF22C2AF207502C29130751C
:10100B0002C295206A0302102C9001F1206C123061
:10101B006E0F207502C295307502C2917428D5E00F
:10102B00FDD293207503759F00307503759F207556
:10103B003D06D2AF22C2AF206A0302106A9003565C
:10104B00306E1F207502C295307502C29120750259
:10105B00C291307502C2957428D5E0FD02106D90D7
:0F106B0001D7207502C294307502C290305A0E20
:10107A00E525600A207502D290307502D294207557
:10108A0003759F20307503759F00753D01D2AF220D
:10109A009001B1C294C292C290C295C293C29122E7
:1010AA00C3E54F9535E55095365001227890E6FF15
:1010BA00C3EF94055018C3EF9404501BC3EF940375
:1010CA00501EC3EF94025021C3EF94015024C3E58C
:1010DA004F943CF8021105C3E54F9428F802110514
:1010EA00C3E54F941AF8021105C3E54F9412F802AA
:1010FA001105C3E54F940AF8021105E5509400F969
:10110A00884F89502230580302110F2278807607BF
:10111A0078817607788276017894760178837604E6
:10112A007886760A788F76037890760178957602B3
:10113A0078927603789B760D789376017887760293
:10114A00789C7601788876017889760178857600A8
:10115A00788C7601788D7600788E76B478967625B6
:10116A00789776D078987678789976C8789A760447
:10117A00789D7600227893E6FF756409756501C348
:10118A00BF02097564057565010211C4C3BF03096D
:10119A007564057565020211C4C3BF040975640547
:1011AA007565030211C4C3BF050675640975650731
:1011BA00C3BF06067564007565007887E6FFC26CD2
:1011CA00C3BF0302D26CC26BC26A7418552D600287
:1011DA00D26AC26E6002D26ED26F6002C26FC275EC
:1011EA007888E630E102D275C2767889E630E10283
:1011FA00D276C3EF94026008758E01D26D02120F87
:10120A00758E00C26D227880E61490008093789ED5
:10121A00F67881E61490008093789FF6119A2278E6
:10122A009BE61490008D9378A0F6119A227886E6B0
:10123A001490009A9378A1F6119A22789CE6149059
:10124A0000A79378A2F6789CE6149000AC9378A352
:10125A00F6119A22227896E6FA7897E6FB30770416
:10126A007A007BFFC3EB9AFCC3948250027C82759E
:10127A006C00056CEC856CF0A4C3E5F0948040F238
:10128A0022C2D353D9BF7581C043FF801207B275FA
:10129A00EF0243B203E5B324044002F5B37580FFBD
:1012AA0075A40075F1DC75D4EF7590C075A53F750E
:1012BA00F23F75D5C075A60175E241119AE4F8F6B8
:1012CA00D8FD3116121823317F5110512951375147
:1012DA0045515E515F7898866D119A758850758967
:1012EA000275C82475910475D8401207C61207D52D
:1012FA001207BE1207DC1207BE1207E31207BE125C
:10130A001CE51207C61207C61207C275A82275B8CD
:10131A000275E69075F610759B80759D0375D10E62
:10132A0075BC5875BB0E75BA1175E8801207B2D232
:10133A00AF120AC443DA01C2D8C2691207C67530AD
:10134A0001D2597A05E55770027A051207B6E558AF
:10135A00C3940240EEE52E541F855A59F55AB559E1
:10136A00E2DAE2C25953DACF20760343DA20307642
:10137A000343DA10C2D8C2691207C21207B678024A
:10138A00741F552E70027800C3E5589840EDC2AF1D
:10139A001207D51207D51207D5D2AF1207C675475D
:1013AA00001207B6788CE6C394015003021474E560
:1013BA0030C394015003021474741F552E6035C350
:1013CA00E55894FF5003021474C2AF1207EAD2AF71
:1013DA001207C2C3E558940150EFC2AF1207D512E3
:1013EA0007BA1207D5D2AF1207C2C3E55894FF4015
:1013FA00E9021D6A7F05D277515F1207C2C2AFC2E6
:10140A0077515FC3E558947FD2AF4068C2AF1207E5
:10141A00EAD2AFDFE1C3E55894057897F61207C61A
:10142A001218D3121CED7F0AD277515F1207C2C27B
:10143A00AFC277515FC3E558947FD2AF50E8C2AFCD
:10144A001207D51207BA1207D5D2AFDFDBE5582447
:10145A00057896F61207C61218D3121D1C1207C277
:0F146A00C3E55894FF40F6021D6AC3E558954745
:1014790040038558471207C2C3E5589401400261E9
:10148900ABC2AF1207EA1207EA1207EAD2AF120794
:10149900C6753000E4F531F5320531E531F47036C1
:1014A9000532789AE67828146012785014600D781D
:1014B900A014600878F0146003753200C3E532980F
:1014C900401415327899866DC2AF1207EAD2AF7807
:1014D90098866D1207C21207B6E5287008741F5561
:1014E9002E7002614BC3E558940640AD1207C2E560
:1014F90028700302134B119AE4F522F523F524F51C
:1015090025755CFF7885865FF53FF540F541F54225
:10151900F543F56AF548F52BF52CF55B120C457585
:101529006A0875BB101207B2120B59E5E820ECFBEB
:10153900A8BDA9BEE97001F8886B120B5D756A0830
:1015490075BB107895E630E00302158F7887E6FEC3
:101559007602317F7887EEF6D261C2AF120C15851B
:10156900225C85225DD2AFC2617525007562007566
:101579006301D260D26375380011021140120CC1A7
:10158900120C450216B17887E6FE76037893E6FDDC
:101599007605317F7887EEF67893EDF6D260D261E1
:1015A900D26E11021140120C151207B2120F041259
:1015B90007B21207B2120F391207B6120F831207B8
:1015C900B61207B6120FC11207BA11021207B612E4
:1015D90007B2C261D262120B59120B5D120C15755A
:1015E9006A0875BB101140120CBA120D3511AA31D7
:1015F9000F120F04120CBA120D3511AA310F120F66
:1016090039120CBA120D3511AA310F120F83120CAF
:10161900BA120D3511AA310F120FC1120CBA120DDF
:101629003511AA310F1102120CBA120D3511AAC3C4
:10163900E54F9535E5509536400C310FC3E5589483
:101649000150930217D9310FC2627887E6FE7602FC
:10165900317F7887EEF685225C855E5D855E25752E
:101669006200756301D263753800C2AF207502C28A
:1016790095307502C291207502C291307502C295EA
:10168900742DD5E0FDD2AF1140120CC1120D1C1200
:101699000D35120DB9756A0075BB0E0216B1317F91
:1016A9001140756A0075BB0E120DDB120E61120E28
:1016B900891208D4120E9D120F04120CC1120D1CAE
:1016C900120D35120DB9120DD2120E61120E8912B8
:1016D9000961120E9D120F39120CC1120D1C120D47
:1016E90035120DB9120DDB120E61120E891209A104
:1016F900120E9D120F83120CC1120D1C120D351200
:101709000DB9120DD2120E61120E891209FE120EB6
:101719009D120FC1120CC1120D1C120D35120DB9FB
:10172900120DDB120E61120E89120A62120E9D1140
:1017390002120CC1120D1C120D35120DB9120DD267
:10174900120B59120E61120E89120B5D120E9D11A8
:1017590040120CC1120D1C120D35120DB930632A3D
:10176900855E5C855E5D756200756301C3E53894CD
:1017790064400AC263D264753714021793C3E558EB
:10178900940140030216B10217D9306419E53714E0
:101799007005C2640216A7F537C3E55894014003E2
:1017A9000216B10217D9C3E55B94014009855E5D54
:1017B9007562FF756301C3E55B94FA5013741F5595
:1017C9002E7004E5286009C3E53C94F05002C1B1CC
:1017D900119A7887E6FE7602317F7887EEF6E4F58E
:1017E90022F523F524F525F55FC2601207B2119A97
:1017F900741F552E7007E528700302134B7895E680
:1018090030E009121CE5121CE5121CE5788DE6C3CF
:101819009401400302138502149D901A0D78201239
:101829001C00E520B4A50CA3121C00E520B45A0342
:101839000218451211161218D30218D2901A0378F9
:1018490080121C00A308121C00A308121C00A30884
:10185900121C00A308A308A308121C00A308121C49
:0F18690000A308121C00A308121C00A308A30868
:10187800A308121C00A308121C00A308121C00A332
:1018880008121C00A308121C00A308A308121C00BD
:10189800A308121C00A308121C00A308121C00A312
:1018A80008121C00A308121C00A308121C00A3089D
:1018B800121C00A308121C00A308121C00A3081283
:1018C8001C00A308121C00901A2122C2AF121C3F50
:1018D800121C19901A00740A121C05A37404121C15
:1018E80005A37410121C05901A037880121C04A317
:1018F80008121C04A308121C04A308121C04A30841
:10190800A308A308121C04A308121C04A308121C91
:1019180004A308121C04A308A308A308121C04A308
:1019280008121C04A308121C04A308121C04A30810
:10193800121C04A308A308121C04A308121C04A365
:1019480008121C04A308121C04A308121C04A308F0
:10195800121C04A308121C04A308121C04A30812D6
:101968001C04A308121C04A308121C04A308121CBC
:0B19780004121C52121C30901A212295
:101A00000A041007070104FFFF0A020101A55A0199
:101A100000B40301FF0301010225D078C8040D01C1
:021A200000FFC5
:101A40002348694D6F64656C436F6F6C323241237C
:101A500023424C48454C4923463333302320202031
:101A60002020202020202020202020202020202076
:101C0000E493F622E6438F01538FFD75EF0275B71B
:101C1000A575B7F1F0538FFE22438F02438F0175F4
:101C2000EF0275B7A575B7F1901A0DF0538FFC222E
:101C3000901A0D74A59105901A0E745A9105227A86
:101C40003079D07820901A409100E520F709A3DA86
:101C5000F7227A3079D0901A40E7910509A3DAF992
:101C600022AB6EA86FBB01057980021CE2BB0205A6
:101C70007981021CE2BB03057982021CE2BB0405E8
:101C80007994021CE2BB05057983021CE2BB0605C0
:101C90007995021CE2BB07057986021CE2BB0805A8
:101CA000798F021CE2BB09057990021CE2BB0A0590
:101CB0007992021CE2BB0B05799B021CE2BB0C056E
:101CC0007993021CE2BB0D057987021CE2BB0E056D
:101CD000799C021CE2BB0F057988021CE27989021B
:101CE0001CE2E8F7227C051207C6DCFB22C2AF1219
:101CF00007D51207DC1207E31207EA1207BA120728
:101D0000D51207DC1207E31207EA1207BA1207D549
:101D10001207DC1207E31207EAD2AF22C2AF1207A2
:101D2000EA1207E31207DC1207D51207BA1207EA14
:101D30001207E31207DC1207D51207BA1207EA12DC
:101D400007E31207DC1207D5D2AF22AE6EAF6FC227
:101D5000AF1207D51207D51207D51207BADEF21255
:101D600007EA1207BADFF8D2AF2291ED91E591E5CB
:101D7000756E01756F01757000B14B7C05AD581221
:101D800007C6C3ED955870F5C3E55894014009C3E3
:101D9000E55894FF4032A1A691611218D391EDC28B
:101DA000AF75EF1291E5DCD50570C3E57094035073
:101DB0000280C691E5056FE56E149000B193F808B6
:101DC000C3E56F98500280AE91E591E5056EC3E5DD
:101DD0006E94115002809C1211161218D3C2AF7566
:041DE000EF1291E588
:00000001FF
